:02000000252BAE
:080008008207473450345334E1
:1000100054347234613463346B3420347634303485
:100020002E343434003482074E346F342034533449
:100030004D345434203466346F3475346E34643443
:10004000213400340339820700346434C8340F3952
:10005000820700340A3414341E34283432343C34D9
:10006000463450345A3407398207243447345034E4
:1000700052344D3443342C34073982072434473406
:1000800050344734473441342C348207003406342A
:1000900001340634013407340134033403340434A6
:1000A00000340634003400340034003401340234A7
:1000B0000034043401348207003400340634073439
:1000C0000D340E341534163419341C3420340034F5
:1000D0002034203420342034203421342334233479
:1000E00027348400B6017928840000082220B60055
:1000F000840A00082720B607840A00080F3936074B
:100100000800B7012721B1202729B5000A3036029F
:100110000318BB28B608031DCA2837083320350644
:10012000031D2729B70A2C303506031D08004F3060
:10013000840030308000840A8000840A8000840AB1
:100140008000840A8000840A8000840A5C30840075
:1001500030308000840A8000840A8000840A800095
:1001600013293930840030308000840A0408613A51
:10017000031DB32808000B3036020318CA283708BD
:100180003C203506031D0800B70A2C303506031D38
:100190000800132935082C3A03191329360845207D
:1001A0003706031908003608073A0319EC28360801
:1001B000083A0319EC283608133A0319EC283508D5
:1001C0002E3A0319080036085B203707393E8400B1
:1001D00035088000B70A080035082E3A03190A29A5
:1001E00036085B20393E8400840A000884038000BE
:1001F000840A840A000884038000840A3608133ABB
:10020000031D0729840A000884038000840A350836
:100210008000080036084520B70008005B20393E02
:10022000840000080800B701B60A3608153A031D15
:1002300008002B21003803191F290614222906144F
:100240008A211A233B21E508031D8A218C22B7014C
:10025000B6010610080002300E21413A031D003499
:1002600010300E21313A0319013410300E21323A88
:100270000319013400344F307420B200B400B301CC
:10028000B20DB30DB20DB30DB20DB30DB20DB30D72
:100290003408B202031CB303F830B205B30CB20C3D
:1002A000B30CB20CB30CB20C4F30840058210800D0
:1002B0002F3080003208800AB20064303202031806
:1002C0005B290008303A203003198000840A2F305F
:1002D00080003208800AB2000A30320203186A290C
:1002E000840A3208303E800008000430EF00E50147
:1002F000E301E40108002B30EE004430E50203186E
:100300008429E5092D30EE006508B2006B308400C9
:1003100058210800EF08031D8E29752193216408D8
:10032000E500EF0308002030EA003630EB0003114F
:1003300000000519E30A0319E40AEA0B9829EB0BFC
:1003400099290800E6000000E60BA429080083169E
:1003500005168511831285110800E8000A30E700B0
:1003600003108511031C85154030851E1E30A22107
:100370000314E80CE70BB12908000D30C62908006A
:100380000A30C62908002030C6290800AD296810A7
:10039000051E00340930E7001430851E0A30A22102
:1003A0000310051E0314E80C4030851E1E30A221E8
:1003B0000000E70BD0296808051ADC29681408003A
:1003C000C721681CE02908007F3983169B001C1494
:1003D0001A08831208007F3983169B008B131C15A3
:1003E00055309D00AA309D009C141C118B179C1841
:1003F000F729831208008316A73081000F3086008A
:100400008312061406220610A3010800A5011E305F
:100410005622303018222030182228304522083049
:100420004522013045220C30452206304522080085
:100430001F220611861086154B2286110800A40083
:1004400025080F39F038A500831686008312861020
:100450000615861506088611861586118039031D36
:10046000272A061125080F39A50083168600831256
:10047000240808001F220611861486154B228611B7
:100480008615A40E4B228611080018228615A40E8C
:100490004B22861108000F308605F03024058604B3
:1004A0000800A530A600A60B532A0800A700512279
:1004B000A70B572A0800C0304522E5080319762A01
:1004C0007B2153303A224D303A2254303A223A308E
:1004D0003A220F236E083A226C083A226D083A221B
:1004E000DF303A2243303A220F230800A0012008CF
:1004F0001320003803197F2A3A22A00A772A08001D
:1005000080304522A00120080420003803198B2ADE
:100510003A22A00A832A08000518942A231C922A4A
:100520002310942A2314942A803045222B2100384A
:1005300003199C2A2A30031921303A222318CB2A86
:1005400003300E213A220B23DF303A220B230B23F8
:1005500012230B230B230B230F2307300E213A22E8
:100560000B230B231523C030452205300E213A22E0
:100570000B230B23DF303A220B230B2312230B23F5
:100580000B230B230F2313300E213A220B230B23B3
:100590000B230B23080000300E213A220B233A30A4
:1005A0003A220B230B233A303A220B230B230F233F
:1005B0000F2307300E213A220B230B231523C030C3
:1005C0004522E5080319EE2AEF0803197B216C0880
:1005D0003A226D083A226E083A22F62A02300E219B
:1005E0003A2210300E213A220F23F62A09300E212A
:1005F0003A220B2312230B230B23122311300E213B
:100600003A220B230F2308300E213A220B230B230F
:10061000DF303A220800840A00083A22080020301D
:100620003A2208002E303A2208004B303A226D3030
:100630003A22080006141F2306101F23080000009A
:10064000A00B1F2BA20B1F2B0800831207309F004B
:100650008B01A7218120FB2175218A218A218A21F2
:100660008A211A231A2380225B227E2B851C602B71
:10067000C721681C362BA0001B3A0319422B200807
:100680008520362BE021A0001B3A0319422B2008BD
:10069000443A0319692B2008553A0319742B200892
:1006A000563A03197E2B2008523A03198A2B200848
:1006B0004D3A0319602B2008723A0319932B362BFD
:1006C00075218A218A218A2106148A2106105B223B
:1006D000362BA001E02183169A0083122008EB211B
:1006E000A00AA01F6A2B362B8030C621A00120084B
:1006F000E421C621A00AA01F772B362BA0012008D9
:10070000042000380319872BC621A00A7F2BBD21A6
:10071000C021362BA001200884000008C621A00AB1
:10072000031D8B2B362B9523362B39308400000884
:10073000C621840A0408613A031D972BBD21C021FC
:020740000800AF
:02400E00020DA1
:024200000000BC
:00000001FF
